:030000000219FDE5
:03000B000200AA46
:03002B0002015C73
:03005B000202EEB0
:030073000202DBAB
:1000800002030406080C10182030406080040608A3
:100090000C10182030406080A0C00003070F1F0D17
:1000A0000D0403060D0503030202C2AFC0D0C0E079
:1000B000206214E5256009E473E525F4F58AD2622F
:1000C000D0E0D0D0D2AF3285268AC262E526F46075
:1000D0002F30682520720DD0E0D0D0D292D291D2AC
:1000E00090D2AF32D292D291D290206F0C2065097B
:1000F000740AD5E0FDE57B4290D0E0D0D0D2AF329B
:10010000758A00C28DD26201F901B9306805206597
:1001100002C29201B9306805206502C29101B9306E
:100120006805206502C29001B9C29330680A206553
:10013000077408D5E0FDC29201B9C29430680A2064
:1001400065077408D5E0FDC29101B9C29530680A0F
:100150002065077408D5E0FDC29001B9C2AFC2ADF9
:1001600053E6EFC0D0C0E0D2D3D2AFC2CEE52A6012
:100170000720744F152A21C37800790020742EE5DA
:1001800080307E01F430E40278FF53DACF207E0322
:1001900043DA20307E0343DA10C2D8C271E58030E2
:1001A0007E01F430E40279FFC3E89970CB3061033B
:1001B000752A40207403752A40885CD270E8600379
:1001C000755F0020740DE52B6004152B21D343DAF5
:1001D00001C2D820700221E6A85C206102C2702012
:1001E000740221E488227882B6040385222420CF79
:1001F0000AD0E0D0D043E610D2AD32C2CF053A7873
:1002000002E52A6005307402152AC3E55C940140BA
:1002100005755F004127756000756900E55F240181
:10022000F55F5003755FFF7982B7020D306E1DC315
:10023000E52294324016854C227982B7030E306E47
:100240000BC3E52294324004798E8722C3E52395BF
:1002500022600840041523415B0523D8CA0569E5DF
:100260006970021569D56A69756A017808E56B607D
:10027000497805C3E569956B4057C3E569956C50AE
:10028000087801756A03020295C3E569956D50050A
:100290007801756A01C3E5629524401E7982B7042E
:1002A0000241C6206E14852462E569046003856BF3
:1002B00069756A0175233C0202D1E5622850057513
:1002C00062FF41C6F562E5620470067560FF7569FC
:1002D000FFD0E0D0D043E610D2AD32C2AF53E67FBC
:1002E0007592FA7593FFC260759104D2AF32C2AFB6
:1002F00053E6EFC2ADC0D0C0E0C0F0D2D3D2AFA8B9
:10030000FBA9FCC2D8307102615553DACF207E03BD
:1003100043DA10307E0343DA20D271E580307E016B
:10032000F420E402612C88278928A13A53DACF20EF
:100330007E0343DA20307E0343DA10C2D8C2713024
:100340007402A1267800E580307E01F430E402A139
:1003500026885CA10E53DACF207E0343DA20307E5C
:100360000343DA10C271206102812E53DACF207E5E
:100370000343DA10307E0343DA20C2D8D2718857A3
:100380008958C3E89555F8E99556F97B007E087AB7
:1003900000C3E8948CE994005005755B00812088C7
:1003A0002178A2E6A8216055C3E894C8E9940050DA
:1003B00008E4D2E4FB7A0A61FBC3E89468E994019B
:1003C0005008E4D2E3FB7A0F61FBC3E894D0E994D0
:1003D000025008E4D2E2FB7A1E61FBC3E894A0E974
:1003E00094055008E4D2E1FB7A3C61FBC3E89498A1
:1003F000E994085008E4D2E0FB7A787E00C3E895DF
:1004000059FCE9955AFD30E70AECF42401FCEDF4BF
:100410003400FD755B00C3EC9AED9E5003755B01E3
:100420008859895A8557558558567802A10EC3E8D0
:100430009527F8E99528F9307C0281F2307B02811A
:10044000F2307A0281EB2075028151E9FDE8FC81EE
:1004500070E9C313F9E813F830790281EBE9C313AB
:10046000F9E813F830780281EBE9C313FDE813FCD7
:0F04700020612CC3EC941CED940240028187EDB7
:10047F00701EC3EC94C850180529E5297002152980
:10048F00C3E529940A5002A126755C00D270A126FB
:10049F00E529600215297400207F037896E624FA77
:1004AF00FEE43400FFC3EC9EFCED9FFD5006780088
:1004BF00790081F2C3EC94FFED9400400678FF7948
:1004CF000081F2EC8572F0A4C5F0A2F733F8790041
:1004DF00400302050E78FF790002050EE9C313F9F8
:1004EF00E813F8307C0EE9600278FFC3E81338F8A0
:1004FF00E43400F9C3E894FFE99400400278FF88E0
:10050F005CD270206102A126741FF4552F4BF52F7A
:10051F00C274EB7002D274752A40307403752A0AC4
:10052F00306102A13A20740353DAFE207403752B55
:10053F0020D0F0D0E0D0D0D2AD43E6103279010216
:10054F00056A790302056A790A02056A791E0205AE
:10055F006A796402056A79C802056A7817E4D5E0FA
:10056F00FDD8FAD9F6227A147B780205917A107B9E
:10057F008C0205917A0D7BB40205917A0B7BC80230
:10058F000591E573D5E001227902E4C294D5E0FD2F
:10059F00C291D5E0FDD291D5E0FDD294D5E0FDE931
:1005AF0020E002C29230E002C290E573D5E0FDE98F
:1005BF0020E002D29230E002D2907496D5E0FDD9BD
:1005CF00C9EAF8D5E0FDD8FBDBB8C29422C37C00A2
:1005DF007D0075F00005F0EA33FAEB33FB50F6EBD4
:1005EF0013FBEA13FAC3E9FFE8FEE89AF8E99BF96F
:1005FF005004EFF9EEF8B3EC33FCED33FDD5F0DF3B
:10060F00EDF9ECF822E889F08A20D2D4F8A9F07B32
:10061F000030F70B7BFFF42401F8E9F43400F9E81C
:10062F008520F0A4ADF0F8E98520F0A4AFF0FEED41
:10063F002EF974003FFA7C04C3EA13FAE913F9E8C0
:10064F0013F8DCF48BF030F70AE8F42401F8E9F43E
:10065F003400F9E889F0C2D4F8A9F0227882B60400
:10066F000302070AC3E55C9419401EE52D5406707A
:10067F0018206E3678057994E7146007780A1460AD
:10068F00027812C3E54198401F306E098564627588
:10069F0069FF756A01852224E4F544F545F546F5B1
:1006AF0047F548C26E02070AD26E7994E7147013A9
:1006BF00E523F43333F913F8E9540104F9E854FE50
:1006CF000206FEE714147014E523F4333333F913E1
:1006DF00F8E9540304F9E854FC020706E523F43360
:1006EF00333333F913F8E954070404F9E854F8C322
:1006FF009440F8E99400F98844894522C3E54113F1
:10070F00F9E54013F8C3E54498F8E54599F9500C1D
:10071F00C3E89480E994FF4016020742C3E8947F30
:10072F00E994005003020742787F7900020742786C
:10073F008079FF8849894A22E5492546F8E54A35F7
:10074F0047F9854A20E4300701F43548FA30E709C4
:10075F00C3EA94F04015020780C3EA940F500302D6
:10076F00078078FF79FF7A0F020780780079007A87
:10077F00F0C3E5249561500AC374019524500B0210
:10078F00079EE54A20E70E02079EE54A30E70688F6
:10079F004689478A482278A5E6FAC3E54933F8E542
:1007AF004A33F9D114E930E70BC3E89480E994FF99
:1007BF004013E1D8C3E8947FE994005002E1D87860
:1007CF007F7900E1D8788079FFE820E715C3E5232A
:1007DF0098F84009C3E8940140030207FF7801022B
:1007EF0007FFE8F424012523F840030207FF78FFF1
:1007FF00884B2278A6E6FAA847A948120614E930D2
:10080F00E70CC3E89401E994FF4016020834C3E8EB
:10081F0094FFE99400500302083478FF790002082E
:10082F0034780179FFE920E715C3E54B98F84009C3
:10083F00C3E89401400302085B780102085BE8F407
:10084F002401254BF8400302085B78FF88242278A7
:10085F00FF20692879A1E76023E541601F74FF85B8
:0E086F0041F0848539F0306A0375F005A4F875
:10087D00C5F0600278FFC3E895645002A8648863F0
:10088D0022C3E5409440E5419401E5635003140112
:10089D009F046002F563227883E6F520120F22751E
:1008AD00E89012054C75E89030EDFDA8BDA9BE127B
:1008BD000FC9756EAF756F00C3740013FD74AF6013
:1008CD006613FC74AF2CFC74003DFDECFAEDFBC31C
:1008DD00E89AE99B4014E56E24AFF56EE56F3400A0
:1008ED00F56FEA2CFAEB3DFB80E5AE6EAF6FC3E51D
:1008FD006F13F9E56E13F8C3E913F9E813F87A03EA
:10090D00C3E913F9E813F8DAF7AA201A7009756E1E
:10091D0000756F000209341AEA6008EE28FEEF39FF
:10092D00FFDAF88E6E8F6F2275E890227883E6FFDE
:10093D0030EDF9A8BDA9BE0570C3E570940840520D
:10094D00757000E9FA79A0E76044EA7007E5716017
:10095D001B02096DC3E895716010E5715006600CBE
:10096D00140209790460F9020979E571F571C394EE
:10097D0058401B7561C0C394044013756180C394C6
:10098D0004400B756140C39404400375610075BB51
:10099D000322EFC39401601F74AF601BC3E894FF83
:1009AD00E994035012C3E8956EE9956F5009E5611E
:1009BD00600C15610209CBE561F460020561A86167
:1009CD00C3E524985002A824C3E89562400AA862A2
:1009DD00E562F4600385626188258826E570B407B9
:1009ED000375BB1022743279A787F0A4C5F0A2F766
:1009FD0033F8C3E895614002A861882288248825D0
:100A0D0088268864227540007541F022C2AF75C8F2
:100A1D0020A8CCA9CDAA3A30CF010A75C824D2AFEF
:100A2D00AB3BAC3C883B893CC3E89BF8E99C206917
:100A3D0008F9306602612A4184AD3D8A3DF9EA9D8F
:100A4D00FA600678FF79FF4169AE3EAF3F8B3E8C71
:100A5D003FA83BA93CC3E89EF8E99FF9C3E54113C4
:100A6D00FBE54013FAE82AF540E93BF541500675E0
:100A7D0040FF7541FF41D1AA40AB41AC40AD417E35
:100A8D00047F02C3EB9404400D1E1FC3EB9408407A
:100A9D0005206A021E1FC3ED13FDEC13FCDEF7C328
:100AAD00EA9CFAEB9DFBEF6009C3E913F9E813F833
:100ABD00DFF7EA28FAEB39FB8A408B4150067BFFC2
:100ACD008B408B41C3EB94025002D2663069047F98
:100ADD000341FC7892E6FFC3E537948240110FC3C2
:100AED00E53794A040010FC3EF940640027F057EC9
:100AFD0002E541C4540FF9E541C454F0F8E540C492
:100B0D00540F28F8C3E89EFAE99400FB4009C3EAA4
:100B1D009402EB940050047A02E4FB6176AA40AB98
:100B2D0041EBC4FEEAC4540F4EFCC3EA9CFAEB94AD
:100B3D0000FBC3E813C313F8EA28FAEB3400FB8A71
:100B4D00408B41C3EB94024002C2667802EBC4FEB7
:100B5D007B00EAC4540F4EFAC3EA98FA4005C394D9
:100B6D000250027A027892E6FF306002617685517A
:100B7D0092855293D26043E680C3E49AF8E49BF9E0
:100B8D003066028102E8FAE9FBD3E913FDE813FCB4
:100B9D0088518952C3EF94036038EF20E00DE82CA3
:100BAD00F8E93DF9ECFAEDFB020BCBE828F8E93951
:100BBD00F9C3E82402F8E93400F97AFE7BFFC3EFAC
:100BCD009403400E8A538B54884D894E8C4F8D5013
:100BDD008136885389548A4D8B4E8C4F8D50306998
:100BED00127553F07554FF754FF07550FF7551F038
:100BFD007552FF8136E8FAD3E813FC8851C3EF94A0
:100C0D00036020EF20E007E82CF8ECFA8122E828B9
:100C1D002402F87AFEC3EF940340088A53884D8C62
:100C2D004F813688538A4D8C4FE568C3335002642B
:100C3D006BF5683060028140753402D26043E68006
:100C4D00E52D54066034A840A941C3E913F9E81312
:100C5D00F8C3E913F9E813F8306904E92440F9C23F
:0E0C6D00AF53E67F759100C3E498F594E499C7
:100C7B00F595759104D26043E680D2AF22D26475AC
:100C8B004300752000306C03752040020CA7D26422
:100C9B00754300752040306C037520007801790195
:100CAB00206620E52D54066002C2647914E541C329
:100CBB0013700104F8C3941440027814306904785B
:100CCB001B791B206010E543600C306903D534049D
:100CDB00D26DA15291480543E59BF45440B52002D7
:100CEB00A13C30690908C3E89940011881CE206402
:100CFB000A08C3E899400281A781CEC264C2AF53F0
:100D0B00E67F7591003066127594007595F87591B4
:100D1B0004D26043E680D2AF81A7E5417EFFC333A7
:100D2B004005C3334001FEC3E49E759400F595A1C5
:100D3B0019C3E5339401500281A730640281A7D80F
:100D4B0002A15081CEC26DC2AF53E67F7591008573
:100D5B005394855495759104854D92854E93D2602D
:100D6B0043E680D2AFE52D54066008206A020533B6
:100D7B00020D8E306D0D206C0A20640715811581D4
:100D8B0002163D2278003064027801E53775F007D2
:100D9B00A4F9E5F028F5F0E9A2F013A2F113A2F201
:100DAB0013F537C394785003753778C3E537953807
:100DBB004008D265D292D291D290306002A1C58503
:100DCB004F92855093D26043E68022207D16C2AFAE
:100DDB00754202C294D293306202C290D2AF759F19
:100DEB0010020FC6C2AF754202C294D29530620296
:100DFB00C292D2AF759F10020FC6307243207D2076
:100E0B00C2AF75420390013A757B10D290C29530F8
:100E1B006204C291C123D294D2AF759F20020FC638
:100E2B00C2AF75420390013A757B10D292C29330D8
:100E3B006204C291C143D294D2AF759F00020FC618
:100E4B00207D17C2AF754203900115D2903062021C
:100E5B00C291D2AF759F20020FC6C2AF75420390ED
:100E6B000115D292306202C291D2AF759F00020F70
:100E7B00C6207D16C2AF754204C293D29530620272
:100E8B00C291D2AF759F00020FC6C2AF754204C2AA
:100E9B0095D293306202C291D2AF759F20020FC6DA
:100EAB00307243207D20C2AF754205900129757BBE
:100EBB0008D291C294306204C292C1C9D293D2AF0C
:100ECB00759F10020FC6C2AF75420590014B757B23
:100EDB0020D291C294306204C290C1E9D295D2AFB4
:100EEB00759F10020FC6207D17C2AF75420590018A
:100EFB000BD291306202C292D2AF759F10020FC615
:100F0B00C2AF75420590011FD2913062EBC290D2F5
:100F1B00AF759F10020FC6207D16C2AF754206C279
:100F2B0095D294306202C292D2AF759F20020FC647
:100F3B00C2AF754206C293D294306202C290D2AF56
:100F4B00759F00020FC6307244207D20C2AF7542E0
:100F5B000190014B757B20D292C293306204C290F8
:100F6B00E16FD295D2AF759F00020FC6C2AF75422B
:100F7B0001900129757B08D290C295306205C2920F
:100F8B00020F90D293D2AF759F20020FC6207D1710
:100F9B00C2AF75420190011FD292306202C290D251
:100FAB00AF759F00020FC6C2AF75420190010BD205
:100FBB0090306202C292D2AF759F20C2652290011F
:100FCB0009757B00D292D291D290C293C294C295F2
:100FDB00C2622278807607087607087601087604C5
:100FEB000876FF0876FF087609087602087601086E
:100FFB007601788C76010876000876B40876FF08BF
:10100B0076FF0876FF0876030876FF0876010876E8
:10101B00FF0876250876D00876780876C808760417
:10102B000876FF08760108760008767A08760A08B3
:10103B0076010876010876000876FF08760022789C
:10104B0087E6FFC272BF0302D2727888C27DE63098
:10105B00E102D27DC27E7889E630E102D27EC3EF17
:0F106B0094026008758E01D27302107C758E009E
:10107A00C273227880E6149000809378A5F678816E
:10108A00E6149000809378A6F67886E61490008D90
:10109A009378A7F6789FE6F87005756B0001C3C3CD
:1010AA00E8941140027811E82828F56B256B256B26
:1010BA0028F56C256B2828F56D7886E6F539C394F2
:1010CA00025003753902789CE67538FFB40203753D
:1010DA0038A0B4030375388278A3E61490009A9373
:1010EA00F566120FC922227896E6FA7897E6FB7817
:1010FA0088E6B40305C3EB940EFB307F047A007BC9
:10110A00FFC3EB9AFCC3948250027C82757200057D
:10111A0072EC8572F0A4C3E5F0947D40F222D27F8E
:10112A0011F112055B12055B7A007B007C10120537
:10113A0051E55C2AFA74003BFBDCF37C04C3EB1335
:10114A00FBEA13FADCF7FEC27F11F122757C007507
:10115A007D00E5EF20E6037520000520903FFFE5BE
:10116A0020146006901DFF1460009304600375EF5D
:10117A001653D9BF7581C043FF8012054C75EF061F
:10118A0043B203E5B3240220E70DF521E5E320E0AD
:10119A00068521B343E301120FC97580FF75A400C8
:1011AA0075F1D475D4EF75908775A54075F2FF7502
:1011BA00D5BF75A60175E24275DB4675EA02120FC4
:1011CA00C9E4F8F6D8FD756801120FDE1216947894
:1011DA00988673753001C2AF12056512057512053E
:1011EA005B12057C12055B12058312055B1217C799
:1011FA00120565120565120560C2AF757C00757D22
:10120A000078FA79FA308407D9FBD8F7021C001162
:10121A004A117D11F011F178988673120FC97588F9
:10122A001075890275C82475910475D84075A8226D
:10123A0075B80275E690759B80759D0075D10E751F
:10124A00BC5875BB0375BA1175E88012054CD2AF4C
:10125A001208A475360053DACF207E0343DA203011
:10126A007E0343DA1043DA01C2D8C271120565D28D
:10127A00617B037A0CE55B70077A0CDB03021203CD
:10128A0012055B207003021203C270E55CC394026C
:10129A0040E1E52F541F855E5DF55EB55DD5DAD573
:1012AA00C26153DACF207E0343DA20307E0343DA69
:1012BA0010C2D8C27178A2E67008D274E52F54E041
:1012CA00F52FC275752900120560307409C3E52926
:1012DA00940A4002D27512055178023074027800DD
:1012EA00C3E55C9840F0C2AF120575120575120588
:1012FA0075D2AF120565754C00120551788CE6C39C
:10130A00940150030213F0E530C394015003021311
:10131A00F0757CA5757DF1207435C3E55C94FF50AA
:10132A00030213F0C2AF12058AD2AF120560C3E5F9
:10133A005C940150EFC2AF1205751205561205757D
:10134A00D2AF120560C3E55C94FF40E902184C7FF6
:10135A0005D27F11F1120560C2AFC27F11F1AE5CF6
:10136A00C3E55C947FD2AF5002810012054CC2AF34
:10137A0012058AD2AFDFDA3128C3EE94057897F6E0
:10138A001205651217CF7F0AD27F11F1120560C2CA
:10139A00AFC27F11F1AE5CC3E55C947FD2AF50E679
:1013AA0012054CC2AF120575120556120575D2AF59
:1013BA00DFD63128EE24037896F6F87997E7C394B6
:1013CA00824003985006E824827897F6120565123F
:1013DA0016E21217FE12056011F1C3E55C94FF5084
:1013EA0002611B02184C757C00757D00C3E55C9593
:1013FA004C4003855C4C12056078017988E7B40398
:10140A00027805C3E55C9840026103C2AF12058AFF
:10141A0012058A12058AD2AF120565753000E4F505
:10142A0031F5320531E531F4703F0532789AE678C4
:10143A0019146012783214600D787D14600878FAF5
:10144A00146003753200C3E53298401D120FC912A9
:10145A00054C153275310078998673C2AF12058A28
:0E146A00D2AF78988673120560120556E52AF7
:101478007005307402410378012074027806C3E5D0
:101488005C9840A1120560E52A7003021203C2AFFE
:10149800120FC9E4F522F523F524F525F526F5679D
:1014A800D2AF7885E6C333F565E4F544F545F546EE
:1014B800F547F548F570F52CF52DF5377570087575
:1014C800BB1012054C12093530EDFDA8BDA9BEE9C7
:1014D8007001F8887112093975700875BB10114AC6
:1014E800C2AF7561FF1209F28522618522628522E9
:1014F80063D2AF7522017524017525017526018512
:101508006069756A017888E6B40307C27D3076029F
:10151800D27DD268D269753300120F22120F511290
:101528000A12120A19120A12120A19120A12120CB3
:101538009912066B120D8F120DD6120A19120C8809
:10154800306E0312070B20660312085E3066031222
:10155800088E120D8F120E05120A19120C99306E90
:1015680003120747120D8F120E7C120A19120C88EB
:10157800306E031207A5120D8F120EAB120A191244
:101588000C99306E03120802120D8F120F22120AE4
:1015980019120935120C88120D8F120F51120939C0
:1015A800120A1930692C85646185646285606975E1
:1015B8006A0179187A0CC3E533994009C269D26A7D
:1015C8008A350215DAC3E55C940140030215360238
:1015D8001645306A25206C22E535147006C26AD299
:1015E8006BA136F535C3E55C9401400302153678E6
:1015F80088E6C394036003021645753600C3E55FA9
:1016080094014009856462856069756A0178FA7990
:10161800A4E760027803C3E55F985021307404E5BD
:101628002A601A78F0306C058564617820C3E5413A
:10163800985002A1360536E55C6002C1487536004F
:10164800C2AF120FC97887E6FE7602114A7887EE94
:10165800F6E4F522F523F524F525F526F565752C30
:1016680000752D00D2AF120560120FC978A4E6608C
:1016780006C292C291C290307406E52A70024103F4
:10168800788DE6C39401400241E08128901A0D78D4
:1016980020121724E520B4A50CA3121724E520B4C2
:1016A8005A030216C2757CA5757DF1120FDE12165B
:1016B800E2757C00757D000216E1901A0378807B44
:1016C8000A121724A308DBF9901A0F788C7B1912D9
:1016D8001724A308DBF9901A2822C2AF1217671241
:1016E8001744901A00740E121729A37409121729A7
:1016F800A37415121729901A0378807B0A121728E9
:10170800A308DBF9901A0F788C7B19121728A30805
:10171800DBF912177A121758901A2822E493F62246
:10172800E6438F01538FFDFFC3E583941C400122DC
:10173800EF857CB7857DB7F0538FFE22438F024338
:101748008F01857CB7857DB7901A0DF0538FFC22E9
:10175800901A0D74A5F129901A0E745AF129227A5B
:101768003079D07820901A40F124E520F709A3DADF
:10177800F7227A3079D0901A40E7F12909A3DAF9EB
:1017880022AB74A875BB01027980BB02027981BBC8
:1017980003027982BB04027994BB05027983BB06F4
:1017A800027986BB07027992BB08027987BB0902D6
:1017B800799CBB0A027988BB0B027989E8F7227CFD
:1017C80005120565DCFB22C2AF12057512057C12F5
:1017D800058312058A12055612057512057C120535
:1017E8008312058A12055612057512057C120583A7
:1017F80012058AD2AF22C2AF12058A1205831205DA
:101808007C12057512055612058A12058312057C8D
:1018180012057512055612058A12058312057C12E7
:101828000575D2AF22AE74AF75C2AF120575120539
:1018380075120575120556DEF212058A120556DF75
:10184800F8D2AF221217CF1217C71217C775740133
:10185800757501757600112D7C05AD5C120565C3A3
:0F186800ED955C70F5C3E55C9401400AC3E55C47
:1018770094FF403702188F1217891216E21217CFFA
:10188700C2AF75EF161217C7DCD10576C3E576949C
:1018970003500280C21217C70575E5741490009FA4
:1018A70093F808C3E57598500280A91217C7121755
:1018B700C70574C3E574940C50028095120FDE12AD
:0A18C70016E2C2AF75EF161217C744
:0319FD000211567E
:101A00000E091507070104FFFF09020101A55A018C
:101A100000B4FFFFFF03FF01FF25D078C804FF01DA
:091A200000FF0A010100FF00FFB4
:101A400023484B696E673335412320202020202016
:101A500023424C48454C4923463333302320202031
:101A60002020202020202020202020202020202076
:101C0000C2AFC2D353D9BF7581C043B20343FF8073
:101C1000752438752503B1DC7529A5752AF175E29F
:101C20004043F11053A4EF75D4FFD2847DFA7803BA
:101C300079E67C10752200752300901DE97B0675FE
:101C400024987525013084028145208408D8FBD969
:101C5000F9DCF781B7308408D8FBD9F9DCF781B714
:101C6000B19CE493A3C39A6004DDC381B7DBDBB10D
:101C70008E6002812E7B08E493FAA3B16FDBF87AC1
:101C800030B16F752200752300B18EEAFCEBFDC305
:101C9000ED94FE400EB18E8A278B28ED30E0048A49
:101CA000828B83B18E7AC270D8C3ED94FE601950D6
:101CB000CEBD002BEC600F7520007521FF7529004B
:101CC000752A000200008100A827A9280809D80465
:101CD000D90281DCB192EA89AAF281CE0D81A3C337
:101CE000ED94035053EDA2E092007AC5C3E58294CF
:101CF00000E583941C508A200010438F02438F011B
:101D00008529B7852AB7F0300029A827A92808090E
:101D1000438F01538FFDD804D902A133C3E58394C7
:101D20001C4003A3A11689AAE28529B7852AB7F02A
:101D3000A3A116538FFC817F7AC1BD030CE493A34A
:101D4000FAB153DCF8B14B817F8181AA22AB23B178
:101D50006FEBFAEA6222752608C3E52313F523E543
:101D60002213F52250066323A0632201D526EAB18F
:101D7000DCB1DC75260AEAF4200102D284300102CB
:101D8000C284B1DCC3134002C201D526EB22B1925A
:101D9000EAFB208402A192308402A197752608AE46
:101DA00024AF25C3EF13FFEE13FEB1E0B1DCC3EAAD
:101DB000133084024480FA30E703632201C3E52331
:101DC00013F523E52213F52250066323A0632201B5
:101DD000D526D9E52265236523F52222AE24AF2539
:101DE0000E0FDEFEDFFCD20122424C48656C6934E6
:071DF000373164F3300601F6
:00000001FF
